:0300000002000EED
:03000300020055A3
:20000B0002002475810F438901D2AFD2A9D28C12005880FE12001B80FBC0E0C0D0758CFFC3
:20002B00758A000508E508B46403750800C395094004C2908002D290E508C3950A4004C2F4
:20004B00918002D291D0D0D0E032050B327440F59074FFF5B07450F50C741EF50D7400F548
:20006B000E7432F50F120080E5B0440FF5B01200BC0200732205810581740178FD12022609
:20008B00F678FD120226E670030200B7E59008F6E654401202517B0012024812025A45F0D2
:2000AB0070030200B4740018F602008C15811581220581E5B0540FF5B078FE120226F6E6FF
:2000CB0054011202517B0012024812025A45F070030200E91201A97401F50E02018478FE52
:2000EB00120226E654081202517B0012024812025A45F0700302010D1201C87402F50E02C1
:20010B00018478FE120226E61202517B0912024812025A45F0700302013CE50C75F000C009
:20012B00E0C0F0120187158115817400F50E02018478FE120226E61202517B0B1202481271
:20014B00025A45F0700CE61202517B0D12024812025A45F0600CE50E75F0007B007C0012E8
:20016B00025A45F07003020184E50D75F000C0E0C0F0120187158115811581227464F59067
:20018B0078FB120226E6240AF509E6F50AE50F75F000C0E0C0F012020915811581227468C0
:2001AB00F590E50D2405F509E50DF50AE50F75F000C0E0C0F012020915811581227454F5D4
:2001CB0090E50D2405F509E50DF50AE50F75F000C0E0C0F012020915811581227458F59015
:2001EB0078FB120226E6F509E62405F50AE50F75F000C0E0C0F0120209158115812278FBCE
:20020B001202268603088604BB0004BC00012279E5A3D9FD1BBBFFF01C80F4C82581C8225C
:20022B00C92581C97A0022D083D082CF2581F581CFC082C08322CF2581F581CF227C00CBB6
:20024B0030E7011CCB2275F00030E70215F02212026D6009E4F5F02212026D60F7E4F5F057
:20026B000422C5F0C39C7003E5F09B22FBE493CB22FCE493FB740193CC22FAE493F9740192
:03028B0093CA22F1
:00000001FF
